:03216100750800FE
:20216700C009858109E582FF24F850028032AE088FF005F07401800225E0D5F0FBFFE50927
:2021870024FDF8E66005EF42068005EFF4FF5206C006C0069000071221CE1581D0068E08B8
:2021A700D00922AF82C007C0079000071221CE1581D0078F0822E4C0E09000041221CE1572
:0721C700819000020221E4F7
:2021CE00C009858109AD84758408E50924FDF8E6F08D84D00922AD84758408E0FE8D848E4F
:0221EE0082224B
:03210000022108B1
:0321640002210352
:052103001222B080FE75
:2021F000C009858109AF82E50924FDF886F005F0EF800225E0D5F0FBFEE50924FDF886048F
:202210007D007408C39CFCE49DFD8CF005F0EF8002C313D5F0FB4EF582D00922C0098581D5
:2022300009AC82AD83AEF0FFE5812408F581E5092405F8E4F608F608F608F6E5092405F890
:20225000C3E69C08E69D08E69E08E69F504CA80908E4F608F608F608F6A80908C3E6943234
:2022700008E6940008E6940008E694005015A80908740126F6E40836F6E40836F6E40836C7
:20229000F680D6E5092405F8740126F6E40836F6E40836F6E40836F680A1850981D00922CF
:2022B0007F03C0071221BDAE82D007BEAA278F82C0071221AAD0077401C0E08F821221F06A
:2022D000AD8215818D079000C8E4F5F0C00712222CD00780CDEEF4F582C0071221AA90009C
:0B22F000C8E4F5F012222CD00780B7E4
:06213700E478FFF6D8FD7C
:202115007900E94400601B7A009022FF780075A060E493F2A308B8000205A0D9F4DAF275F0
:02213500A0FF09
:20213D007800E84400600A790075A060E4F309D8FC7800E84400600C7900906000E4F0A3E2
:04215D00D8FCD9FAD7
:0D2108007581091222FBE5826003022103AC
:0422FB0075820022C6
:00000001FF
